:020000000F28C7
:10000800FE00030EF1000408F2000A08F300831250
:100018007F08F400882BBB2B8312A100A001512874
:100028005330A4008330A5005C284730A4008330F7
:10003800A5005C284E30A4008330A5005C28F03071
:10004800A4008230A5005C281030A4008330A500ED
:100058005C287B30A4008230A5005C284730A400CF
:100068008230A5005C282E30A4008330A5005C28CF
:10007800CF30A4008230A5005C281230A400823062
:10008800A5005C28AD30A4008230A5005C284E3065
:10009800A4008330A5005C285C2821088400103067
:1000A800040203184B2803308A00AB30040782008F
:1000B8002508FF00240884000022F5007508A20026
:1000C8000130A4070318A50A0030A507A901D429FF
:1000D8002508FF00240884000022F5007508A30005
:1000E8000130A4070318A50A0030A5079E28403050
:1000F800F5007508A600BB282030F5007508A60095
:10010800BB281030F5007508A600BB280830F5009C
:100118007508A600BB280430F5007508A600BB28A2
:100128000230F5007508A600BB28A6010314A60D29
:10013800BB28BB282308E039F500F6017608003A09
:100148000319A72899287508203A03197B28603ACB
:1001580003198028203A03198528E03A03198A28C8
:10016800203A03198F28603A0319942899282608F9
:10017800F5007508A800A029EE3083169200073014
:1001880083129200B729E130831692000730831258
:100198009200B729D4308316920007308312920058
:1001A800B729C83083169200073083129200B72906
:1001B800BD3083169200073083129200B729B230FF
:1001C80083169200073083129200B729A83083164D
:1001D8009200073083129200B7299E30831692004E
:1001E800073083129200B7299630831692000730A1
:1001F80083129200B7298D3083169200073083123C
:100208009200B72985308316920007308312920036
:10021800B7297E3083169200073083129200B729DF
:10022800763083169200073083129200B729703017
:1002380083169200073083129200B729693083161B
:100248009200073083129200B72963308316920018
:10025800073083129200B7295E3083169200073068
:1002680083129200B72959308316920007308312FF
:100278009200B729543083169200073083129200F7
:10028800B7294F3083169200073083129200B7299E
:100298004A3083169200073083129200B7294630FD
:1002A80083169200073083129200B72942308316D2
:1002B8009200073083129200B729FC30831692000F
:1002C800053083129200B729EE308316920005306C
:1002D80083129200B729E130831692000530831209
:1002E8009200B729D4308316920005308312920009
:1002F800B729C83083169200053083129200B729B7
:10030800BD3083169200053083129200B729B230AF
:1003180083169200053083129200B729A8308316FD
:100328009200053083129200B72983169201073094
:1003380083129200B729B72923081F39F500F6015F
:100348007608003A0319A92999297508FF3E031C64
:10035800992984001F3004020318992901308A0062
:10036800E030040782002208F5007508A7007D30F8
:1003780081008B1683161208F5000310750C831282
:1003880093000C3095008B17CB296400CB2983127E
:100398002908031DD029C9298B139501A901D4293E
:1003A8002508FF002408840000220038031DDD29E9
:1003B800DE296C28DF290800C028C728CE28D528C0
:1003C800DC28E328EA28F128F828FF2806290D293F
:1003D80014291B2922292929302937293E29452969
:1003E8004C2953295A29612968296F2976297D2999
:0603F80084298B299229E3
:10040000FF1B0A2A83137F1883170008840A031925
:10041000FF0A08007F087F398A000408840A03194C
:10042000FF0A82002634A6348634A8346A34603445
:10043000AA348A34A83486348334A33460348634AE
:10044000A8348A34AD348D34AD348F34AF348D3428
:10045000AD3468346034A0348D34AA348D34AD3476
:100460008D34AD348E34A0348E34AE3491348F3428
:10047000AF346A348034A8348A34AD348D34AD342A
:100480008A34AA348834A8348634A6340034263416
:1004900082348234A23447344E348B34AA348934C3
:1004A00053346E348B34AA34893453346E348B34E1
:1004B000AA348B34493482348234A23447344E34E3
:1004C0008B34AA34893453346E348B34AA3489344F
:1004D00053346E348B34AA348B3449346234A234AE
:1004E00044348E348B348A3489348734A734893445
:1004F000AA346934003430346D348D34AB34AD34C7
:10050000AF34AD34AB34AA348D34AD34AA346D3449
:100510008D34AB34AD34AA34A834A534A634483471
:10052000A834A634A534A334A534A634A834AA34F8
:1005300068346834A834AA34AB34AA34A834A63456
:10054000A534A334A534A33481348134A134A33435
:100550008534863463344834003413348434A53409
:10056000603480348734A834603480348434A534D3
:10057000A034C0348734A834A034C0348D348B34D4
:10058000C0348534A834A034C0348B344A34A03409
:10059000C034AA3488348534A3348534003411340B
:1005A00079347934763477349634773474346034EB
:1005B00079347934763497349634803474346034B2
:1005C00071347134743472349134723499348D349A
:1005D0008F347134913491348034913474340034D4
:1005E0002334913491349134913491349134A5343D
:1005F000AA34AD34B1349034903490349034903483
:100600009034A634AA34AD34B0346F348D348A3487
:100610008D346D344A34CA34CD34D13496340034F8
:10062000263468348A34AA34A834A034A8348D34EB
:100630008834863468348F34AF34A834A034A83476
:1006400090348F348A3488348F349434A834A63468
:10065000A034A63483348A344834003420349534AA
:10066000913495349A34763460349334903493349E
:100670009734753493349134603491348E347334B8
:100680006E346034933491347534733400341034E0
:10069000CD34CE34CF34CE34CD3400341034813424
:1006A0008034813400341034D93400348B01073065
:1006B0008312990083169101831295018316850197
:1006C0008312850107308316870007308312870065
:1006D0008230831681006C2B83120718702B712BCC
:1006E000742B00301020742B83128718782B792BF1
:1006F0007C2B013010207C2B83120719802B812B3F
:10070000842B02301020842B64006C2B6C2B0F2860
:100710000B117D3081000130A802031D902B912B1D
:10072000A02B2608F0007008A8000130A702031DC6
:100730009A2B9B2BA02BA9010314A90DA02BA02B56
:100740007408FF0073088A0072088400710E830029
:10075000FE0E7E0E0900142819281E284B284B284F
:100760004B284B284B28232828282D283228372887
:100770003C2841284628A601A701A801A901830118
:02078000562BF6
:02400E00C9F3F4
:00000001FF
